:10000000FF23831690003B280528A000030EA100C3
:100010008B12053081000B11A80B11281720073017
:10002000A800210E8300A00E200E8B16090064008C
:100030002708A900051621200000A90B1C2805127D
:100040000034F830A4000000A40B23280034013051
:100050009F000730A300A30B2B289F140730A30099
:10006000A30B30289F1832281E08A50083161E08EF
:100070008312A60000348316D23081000930850037
:10008000831207309900831631309F00831281015B
:10009000A201A301A401A501A601A7010730A800A0
:1000A000A9010512053081000B118B168B17640016
:0800B00027202508A7005728AE
:084000000000010000000000B7
:02400E00CC3FA5
:00000001FF
